:020000004E2B85
:080008009000030E91000A08AC
:1000100092000A108A1083121708161896183E309C
:10002000810213089407131C18281608332094071C
:10003000140C8F003F398F1A403C55200F1B103C89
:100040008F000608F0390F048600960B2B28150840
:1000500093008E1496160B1112088A00110E83005D
:10006000900E100E09008207FF340034FF34003474
:100070000034FF3400340034FF3400340034FF34E3
:1000800000340034FF3400340034FF3400340034D2
:10009000FF3400340034FF3400340034FF340034C3
:1000A0000034FF3400340034FF348207083408344D
:1000B0000934093409340A340A340A340B340B3451
:1000C0000B340C340C340C340C340D340D340D342E
:1000D0000D340E340E340E340E340E340E340F3410
:1000E0000F340F340F340F340F340F340F348B01AF
:1000F0008316F0308605013096008B128316573038
:10010000810083128B1308000C30F4229700083012
:10011000950083165830810083128B168B170800C8
:100120008E1C90281508031C173C95008E100800A3
:100130008207543469346E347934543472346134FF
:100140006B342034763431342E3434340034033973
:10015000820700346434C8340F39820700340A340B
:1001600014341E34283432343C34463450345A3437
:100170000739820724344734503452344D344334E1
:100180002C340739820724344734503447344734F9
:1001900041342C34820700340034013406340134F5
:1001A000073401340334033400340034063401349A
:1001B0000734013401348207003400340034013440
:1001C000073408340F34103413340034003401344D
:1001D000073408340F34003482078634A2344034A4
:1001E00040344034403460343E3454345434313438
:1001F0002E3434342034840099010329840000080B
:10020000A7209900840A0008AC209907840A0008F6
:100210000F39190708009A011A08323E84001A089B
:10022000EC2080009A0A1A080E3A031D0C29882136
:100230002C218829980009301906031936299908B4
:10024000031D43291A08B8201806031D36299A0AE7
:100250002C301806031D08002C308400303080003C
:10026000840A0408323A031D2E297D291A08C12068
:100270001806031D8829093099009A0A2C3018069F
:10028000031D08007D2918082C3A03197D29180838
:100290002A3A031988291908CA201A0603190800DE
:1002A0001908073A031964290F3A03196429180831
:1002B0002E3A031908001908DB201A071C3E840097
:1002C000180880009A0A080018082E3A031979299C
:1002D0001908DB201C3E8400840A00088403800087
:1002E000840A840A000884038000840A18088000B5
:1002F00008001908CA209A0008009A01990A1908EA
:10030000093A031987291908103A031D08008B219F
:100310009A01990108001C3084002730B9000008B8
:10032000413A03199629703A031D98296030B900A3
:100330009B01840A9A01000D990015308407190861
:100340001E3960388000EC3084079A0A1A08063A91
:10035000031D9B290630F4229A00C0301A1CB406F3
:100360009A1CB3061A1DB206A319B5062418B606C0
:10037000AB18B7060730F4223038B8000310B80DB8
:100380002530FB201C3EBA002730FB201C3EBB0062
:100390002930FB201C3EBC002C30FE20BE00BD01DD
:1003A0000A30BD0ABE020318D129BD033E07AC20A6
:1003B000BE006C30BD072F30840000080F39203E8E
:1003C000BE073030FB201C3EBF0027080F393C30F1
:1003D0000319BB0725080F39031D08005030BA0761
:1003E000B61B08000A30BA07B61736130800C30D4B
:1003F000430C902043091F39031D08000310F729FF
:100400000030032A7E30C1000830C200C10CF72141
:10041000C301C20B062A08000130F422C000080004
:100420000A30F422C000080084200022C00B152AE4
:100430000222FF30C400C5000800C1000830C2001D
:10044000410C01300318C5060310C40CC50C031C75
:100450002D2A0830C5068430C406C10CF721C20B12
:10046000202A0800FF30C5064406C00045081D22AA
:1004700040081D22022202227D200800C600000042
:10048000C60B402A080083160516851183128511B4
:100490000800C8000A30C70003108511031C851529
:1004A000A9303E220314C80CC70B4D2A08000D309A
:1004B0005C220A305C2A2030492AC900490E612298
:1004C00049080F39093C031CF93E393C492A4810B8
:1004D000051E00340930C70038303E220310051EC7
:1004E0000314C80CA9303E220000C70B6E2A48082E
:1004F000051A782A481408006722481C7C2A08003C
:1005000083168510051083120130CC00CB00FF301C
:10051000CE009B00CD00CF010800061ECD014A0889
:100520000102CA07031C08000310861E0314CF0D26
:10053000CB0B08002630CB00CD0A0319CD03061ED5
:10054000CD019B0A03199B03CC0B08000A30CC0099
:10055000CE0A0319CE0308008D22CD080319BA2A4A
:100560000530F4224D02031CB72A0510BB2ACB1E0E
:100570000510CB1A05141B08053C0318C62A851064
:100580003908603A27300319B900D02A3908603A8F
:100590000319CF2A4B1A85144B1E8510D02A8514B7
:1005A000CF08031DDF2A0230061F0B30F4224E0253
:1005B000031CDF2A0530F4224D020318EF2A0B300A
:1005C000F4224E02031CF32A4F1805154F08FE3A79
:1005D000031DF32A1022CE018821CF0101340C2201
:1005E000CE018821013400343F3989008316081474
:1005F0008312080808003F39890083168B130815F9
:1006000055308900AA308900881408118B17881882
:10061000072B8312080005151422323084000008CD
:100620001D22840A0408393A031D0F2B0030F422DE
:100630008D000D08F42200380319212B1D228D0A8C
:10064000192B00081D22840A0408403A031D212B9F
:100650000830F4221D220930F4221D228C0B3E2B7F
:100660000330F4228C000430F4228D000D08F422B3
:10067000003803193E2B1D228D0A362B322205111C
:100680000800851405144823851005104823080028
:1006900000008D0B482B970B482B080043220B21A1
:1006A00077208022831605118312051141234123EF
:1006B000412301308C009C2B6722481C652B8D0048
:1006C0001B3A03196A2B0D081A21AC220038031DAE
:1006D0000B235C2B7C228D001B3A03196A2B0D081F
:1006E0000D08443A03198A2B0D080D08553A0319D1
:1006F000942B0D08563A03199C2B0D08313A031917
:10070000A62B0D08323A0319A92B0D08333A031909
:10071000B32B5C2B8D017C2288000D08FB228D0AF7
:100720000D1F8B2B80225C2B8D010D08F4225C2287
:100730008D0A0D1F952B5C2B8D010D08982000381C
:100740000319A52B5C228D0A9D2B5C2B051584209B
:10075000AD2B05158420031090206722481CAD2B7B
:100760007D2005115C2B0515842003109020672245
:06077000481CB52BB02B64
:02400E00F23F7F
:104200000D0028000C0003001E0003000000000049
:104210003E002F000A0003003C009C009E00860028
:104220008200980098006000A4008A009800820034
:10423000B200400061000300F000000020005400C4
:1042400069006E0079005400720061006B0021006B
:0242500000006C
:00000001FF
